:020000040000FA
:1000000049295D2903329E328231042A20003016AC
:100010003D0010186C29901D08000F0887009011F2
:1000200020007839031D983207196B322008343AC2
:10003000031D5F32A001A401B201B013B81BB017B9
:100040003908FB3E03193C32090B0C323B0B0432DE
:100050009630B10012302B32090B4432A830B10077
:10006000433025320903090B063230080139B43E0A
:10007000B10001301C32090B06323A08B0000830DA
:10008000DB20AC001D32E93E031D07323D000E129D
:100090002000A413A50100301A32090B0432F530F8
:1000A000B10007300432090B1D32B0140730B20022
:1000B000BF08031D05323E02031802323E08B2009B
:1000C0003D000E122000B81F09328D2048307C20E0
:1000D000240940390838A400A4170800A413A50176
:1000E0000C30F5333D000E1220000C306B200C302C
:1000F0000332200940390838A0000830A100A017B9
:100100000800B01F02328D20E3333908053A031D81
:1001100008003A083D0096000800A501B20803193E
:10012000080031088400813085003830860087015E
:10013000A519053212001E00A50AB20BF9330408F6
:10014000B10008002000AC1BFE33AD002C09403983
:100150000838AC00AC170800071A0800071D043265
:10016000B01AAC1B080001002908301E033202221D
:1001700080311D3203191B323013E020301F13323F
:100180008700850060308400230015140000000003
:1001900013081A0014081A00910A870BF63340302E
:1001A000A220030103322100B0000130A220200070
:1001B000280940390838A8004030A900A817483459
:1001C0004108870040088600A90B0532523A031DFA
:1001D0000234B0160134A90B023201080800A90B41
:1001E0000332420881000134A90B1C32230095011F
:1001F00007089200871B15170608910020001F3979
:10020000031D02344208B3004308523A031D023270
:1002100030172034173A031D013423001516151525
:10022000412101343C30A906031D023420308400F2
:1002300085003308860023009516151520308700A9
:1002400012008607930012008607940087030319A3
:1002500003324121910AF43395128608031D0334B9
:100260004121871615140000000011001402031D1F
:10027000043411001302031D04349103870BF2337D
:10028000013455309600AA30960095140000000005
:100290000800840182308500210000090319093219
:1002A0009618023296149615961D0332200082315C
:1002B000002A96155D210820FE332100FC309900AC
:1002C0001A095139031DFC33270090309B006C2123
:1002D0003D008E018E1508003D0090011430910004
:1002E000850120308400860003011A00860BFD334F
:1002F0003D000E1796010E120E13901D0332901141
:100300004821FB33163098001E3099001A309A00AD
:1003100020001830A200A6002030AA006030AE00F5
:100320002030A300A700AB00AF00772812340134BF
:10033000003402340234003400340834D834043435
:10034000DA34EF3401340034003400340034013442
:10035000093402344334003402340134003480342C
:1003600032340934043400340034013402340234A9
:10037000013400340534243400341034013404349E
:100380002434023402340534243406340034013475
:100390000534243401340334013407340534823401
:1003A0000334083400340234093404340134003492
:1003B00002340A3400340034003407340534013484
:1003C00002344034003400340734053481340234BC
:1003D000403400340034A13420340034003400347C
:1003E00000340234003403340034803425340034C3
:0803F00000340034003408342D
:020000040001F9
:02000E00CC3FE5
:02001000CE3FE1
:00000001FF
